S01B00006275696C642F6D69636132646F742F6D61696E2E73726563E3
S11300000C945F010C947C010C947C010C947C0195
S11300100C947C010C947C010C947C010C947C0168
S11300200C947C010C947C010C947C010C947C0158
S11300300C947C010C947C010C947C010C94AE0B0C
S11300400C947C010C947E010C94D1010C947C01E1
S11300500C94FB010C9457070C947C010C947C01C8
S11300600C947C010C947C010C947C010C947C0118
S11300700C947C010C947C010C947C010C947C0108
S11300800C947C010C947C010C947C01001C005E9B
S113009000FA017301EA04BC0A5E050202020202CC
S11300A002000000140055008700B901E5043D007A
S11300B0080808080808AEEFEFEFEFEFEF000021A3
S11300C010422063308440A550C660E7700881293F
S11300D0914AA16BB18CC1ADD1CEE1EFF1311210D7
S11300E00273325222B5529442F772D6623993188F
S11300F0837BB35AA3BDD39CC3FFF3DEE3622443E3
S11301003420040114E664C774A44485546AA54BDE
S1130110B528850995EEE5CFF5ACC58DD553367276
S11301202611163006D776F6669556B4465BB77A2E
S1130130A719973887DFF7FEE79DD7BCC7C448E502
S1130140588668A7784008611802282338CCC9ED7E
S1130150D98EE9AFF9488969990AA92BB9F55AD416
S11301604AB77A966A711A500A333A122AFDDBDCCE
S1130170CBBFFB9EEB799B588B3BBB1AABA66C8722
S11301807CE44CC55C222C033C600C411CAEED8F1E
S1130190FDECCDCDDD2AAD0BBD688D499D977EB6B6
S11301A06ED55EF44E133E322E511E700E9FFFBE6E
S11301B0EFDDDFFCCF1BBF3AAF599F788F8891A941
S11301C081CAB1EBA10CD12DC14EF16FE18010A118
S11301D000C230E3200450254046706760B983981C
S11301E093FBA3DAB33DC31CD37FE35EF3B1029068
S11301F012F322D2323542145277625672EAB5CBE8
S1130200A5A89589856EF54FE52CD50DC5E234C3B7
S113021024A01481046674476424540544DBA7FABB
S1130220B79987B8975FE77EF71DC73CD7D326F207
S1130230369106B01657667676154634564CD96D07
S1130240C90EF92FE9C899E9898AB9ABA944586557
S11302504806782768C018E1088238A3287DCB5C5B
S1130260DB3FEB1EFBF98BD89BBBAB9ABB754A54A7
S11302705A376A167AF10AD01AB32A923A2EFD0F27
S1130280ED6CDD4DCDAABD8BADE89DC98D267C07F7
S11302906C645C454CA23C832CE01CC10C1FEF3EFB
S11302A0FF5DCF7CDF9BAFBABFD98FF89F176E3647
S11302B07E554E745E932EB23ED10EF01E00112474
S11302C01FBECFEFD0E1DEBFCDBF11E0A0E0B1E0B3
S11302D0E4E0F5E200E00BBF02C007900D92AC34FD
S11302E0B107D9F713E0ACE4B1E001C01D92A8391D
S11302F0B107E1F70C9448020C9400001F920F928E
S11303000FB60F9211242F933F934F935F936F93E4
S11303107F938F939F93AF93BF93EF93FF939FB17B
S11303208091AD028FB9892F0E941808FF91EF9137
S1130330BF91AF919F918F917F916F915F914F91F9
S11303403F912F910F900FBE0F901F90189526EE9E
S11303508091880390918903A0918A03B0918B03C3
S11303600097A105B10589F080FF0FC080910A03B1
S113037090910B03A0910C03B0910D03863E91055F
S1130380A105B10514F420910A038FB7F8949927B5
S11303902093560321BF109242038FBF0E94F80698
S11303A008951F920F920FB60F9211242F933F932B
S11303B04F935F936F937F938F939F93AF93BF9369
S11303C0EF93FF935F9B06C08CB140E050E060E088
S11303D00E94EB0BFF91EF91BF91AF919F918F9191
S11303E07F916F915F914F913F912F910F900FBE2D
S11303F00F901F90189578941F920F920FB60F923A
S113040011242F933F934F935F936F937F938F9315
S11304109F93AF93BF93EF93FF930E944B0EFF9173
S1130420EF91BF91AF919F918F917F916F915F9168
S11304304F913F912F910F900FBE0F901F901895E1
S1130440AC018FB7F894282F3327E09113038091E0
S113045013038F5F8093130380911303877080933A
S11304601303909113038091CF02981759F02FBF73
S1130470FF27EE0FFF1FEA56FD4F4083518381E0B3
S113048090E00895E09313032FBF80E090E0089577
S1130490C5EED0E1DEBFCDBF1ABA17BA11BA92E0E9
S11304A092B993B9D29AD09AD19A8B9880916100DB
S11304B08F77809361001798A79AA69AA59AA49A11
S11304C0A39AA29AA19AA09A8D9A8F9A8E9ABB986F
S11304D0BF98159AD79AD39A1D9ADF9ADA9A9F5F92
S11304E09C5F9739E8F390E08AE08093B0019093A1
S11304F013039093CF0223EB31E0F9013496ACE47B
S1130500B3E01082BB962D933D939F5F255D3F4FD3
S11305109530B8F3109285031092140310921B03C4
S113052087E193E09093D1028093D00210928603E6
S11305300E942A068FB7F8949927109244038FBF1C
S11305408FB7F894282F332711E01093AD0182E080
S113055080934C0187ED92E09093160380931503EA
S11305601092DB0282E290E090930F0380930E03DB
S113057010929302109291031092900310929002A1
S113058010928F021092A8021092A7021092AB014F
S11305901092A901109266038FEF9FEF9093460388
S11305A08093450390934803809347031092040378
S11305B010924B03E6EBF0E08491992790930303A8
S11305C0809302032FBF8FB7F8949927B998BB98EB
S11305D0BA986B986A986F9A6E9A8FBF17988D9A8B
S11305E08E9A8F9A959A979A969A6AE38091DB02EB
S11305F00E946E066BE380E00E946E0680ED97E039
S11306000197F1F780E88093B902682F8BE00E948C
S11306106E0680E98093BB02682F84E00E946E0618
S11306201092BD028FE68093BE0285E58093BF02DF
S11306306091BD028FE00E946E068091BE02682F19
S113064080E10E946E068091BF02682F81E10E94C2
S11306506E061093C102612F83E10E946E0610930F
S1130660CC0219821A821B821C8220E030E040E016
S113067050E02D833E834F835887BA01A9014987EF
S11306805A876B877C876FEF7FEF8FEF9FE76D87CC
S11306907E878F87988B198A1A8A1B8A7B897C8B21
S11306A083E091E08D8B9E8BA7E2B1E0AF8BB88F96
S11306B0E0E0F0E0E98FFA8FAD89BE89AD90BD909E
S11306C0CD90DD90AD8BBE8BEE24FF248701170106
S11306D0280160E070E885E497E6A60195010E9490
S11306E06012DA01C90181709070A070B070892B1A
S11306F021F02F5F3F4F4F4F5F4F21FF0BC0212C45
S1130700A0E23A2E412C512C8601750116950795CD
S1130710F794E794E2E05695479537952795EA953F
S1130720D1F7DA01C9017EE0880F991FAA1FBB1F08
S11307307A95D1F7820D931DA41DB51D212C60EE71
S1130740362E6FEF462E6FEF562E280E391E4A1E98
S11307505B1E80509042A044B04080509C49AF4BF7
S1130760B04008F060C0AF89B88D8D919C91AA27E4
S1130770BB2742013101681A790A8A0A9B0AD4010B
S1130780C30180509040A044B04080509C49AF4B7E
S1130790B04008F048C0CA01B901A60195010E9401
S11307A03512DC01CB01E80EF91E0A1F1B1F20E1E4
S11307B036EB4DEF5FEFE20EF31E041F151FD80159
S11307C0C70180519641AF4CB941B7FF07C0B095FE
S11307D0A095909581959F4FAF4FBF4F4D855E85F6
S11307E06F85788984179507A607B707E4F42D82E7
S11307F03E824F82588669867A868B869C86E982F9
S1130800FA820B831C83298D3A8D275C3E4FF901B4
S113081020813181298B3A8BFC89FA5FFB8B8D8790
S11308209E87AF87B88B2C892F5F2C8B498D5A8D6F
S11308304E5F5F4F498F5A8F6F89788D6E5F7F4F00
S11308406F8B788F293008F437CF7B89772309F4AD
S113085060C08D818093B1022D813E814F81588586
S1130860BB27A52F942F832F8093B002CA01AA27F8
S1130870BB278093AF0239853093B40249855A85EA
S11308806B857C85BB27A72F962F852F8093B3027A
S1130890CB01AA27BB278093B20259895093B60291
S11308A069897A89872F99278093B50289819A81EA
S11308B0AB81BC818030E5E69E07EDECAE07EDE14F
S11308C0BE07A8F480509448A74DB74128F484E8A3
S11308D08093B70281E904C084E48093B70281E87D
S11308E08093CB0282E08093B80280E70AC08CE850
S11308F08093B70283EF8093CB0282E38093B802A4
S113090080E28093C0022B89220F220F220F2093B2
S1130910BA0249815A816B817C8140938C03509344
S11309208D0360938E0370938F0311E06FEAE62EBC
S113093062E0F62ED7018D917D01682F812F0E94F0
S11309406E061F5F1D30B0F38091C002682F82E1F4
S11309500E946E0660E08BE00E946E066FE382E404
S11309600E946E0661E180E00E946E0666EA8EE0F7
S11309700E946E068EE00E94920683FFFBCF66E221
S11309808EE00E946E0661EE80E00E946E06809109
S1130990CB02682F89E00E946E0660E08BE00E9423
S11309A06E0666EA8EE00E946E061EE0812F0E94AB
S11309B0920683FFFACF66E2812F0E946E0680E9D9
S11309C08093BB02682F8DE00E946E068091CC025A
S11309D0282F33278FB7F894992720937E038FBF4E
S11309E00E94C5068FB7F8949927109270038FBFA1
S11309F08FB7F89499271092970310929603109248
S1130A006F0310926E031092D5021092D4028FBF1E
S1130A100E94C5068FB7F894992716B917B88FBFE7
S1130A208FB7F894482F5527209100013091010188
S1130A3081E597E3289FF001299FF00D389FF00D81
S1130A401124CF018F5A984C9093640380936303CD
S1130A50909394038093930385E89FE0289FB001CB
S1130A60299F700D389F700D1124CB018B57904F27
S1130A709093B2018093B1014FBF109288031092FA
S1130A80890310928A0310928B03109242038FEF12
S1130A90809392038093A7011092940283E0809341
S1130AA0430396EE909356038FB7F894482F552737
S1130AB087B78E7F87BF87B78D7F87BF80B78860F2
S1130AC080BF8BE083BF12BE91BF87B7826087BFB0
S1130AD04FBF30938403209383038FB7F8949927EF
S1130AE010926B03DA9AD89AD99A8FBF0E942A0679
S1130AF0109290008CE089B98CB11BB876E07093A9
S1130B00950088ED8AB98FB7F89499276091AD0163
S1130B108FBF613009F06CC08FB7F894482F552708
S1130B20E0911503F0911603148282E08093AD01E5
S1130B301092A9011092AB018FEF9FEF909346039F
S1130B4080934503809104039927880F991FFC0122
S1130B50E457FF4F24913327322F222783579F4F87
S1130B60FC0184919927282B392B30938E022093F2
S1130B708D024FBF10914B031123D1F46BE3812FEE
S1130B800E946E0680ED97E00197F1F769E3812FEB
S1130B900E946E0688EC90E00197F1F7BB98BA9832
S1130BA00E94E00680EC8DB9B8980E94F80620C037
S1130BB0812F9927880F991FFC01EF55FF4F24912E
S1130BC03327322F22278E559F4FFC01849199277A
S1130BD0282B392B8FB7F89499277093AD018FBFC9
S1130BE0C901AA27BB279C01AD0180E00E940A0726
S1130BF078949091CF0280911303981719F480E0B0
S1130C0090E01FC08FB7F894282F33279091CF021C
S1130C108091CF028F5F8093CF028091CF02877043
S1130C208093CF02E92FFF27EE0FFF1FEA56FD4FF7
S1130C3080819181108211822FBFFC01099581E08E
S1130C4090E08823B1F685B7806285BF889500005F
S1130C500000CFCF8FB7F894682F80E090E04FE486
S1130C6051E09C01F901E80FF91FE95AFC4F448354
S1130C70558312821382118201962B5F3F4F455D8B
S1130C805F4F8230910574F310927D03109211032B
S1130C90109210031092AF011092AE0110924E0107
S1130CA010924D011092A6011092A50110927C039E
S1130CB01092490310927F0310928C0210928B02BF
S1130CC01092AA021092A90280915B0390915C0396
S1130CD090936903809368036FBF0895880F959874
S1130CE096E087FF02C0979A01C097989698969AC3
S1130CF0880F915097FFF5CF979A9698969A959A60
S1130D0097E067FF02C0979A01C097989698969AC1
S1130D10660F915097FFF5CF959A979A969A81E02E
S1130D2090E0089590E0880F959826E030E087FFE2
S1130D3002C0979A01C097989698969A880F215066
S1130D40304037FFF4CF27E030E097989698969A92
S1130D508F98959A969840E050E0879941E0892FC2
S1130D60992721503040442329F0880F991F982F48
S1130D70916002C0982F990F969A37FFEBCF959AFE
S1130D808F9A979A892F992708958FB7F894282FC7
S1130D9080918A02882391F480E090E0E0E7F3E018
S1130DA0819301968C309105DCF38EE180937A0374
S1130DB08FE180937B0381E080938A022FBF0895A3
S1130DC01F9310E061E1812F0E946E068091B702AB
S1130DD0682F89E00E946E06612F8BE00E946E06E8
S1130DE08AEF90E00197F1F781E090E01F91089578
S1130DF080914B01882329F48FE390E10E94200223
S1130E0006C085B7837E85BF85B7806285BF80E0D5
S1130E1090E00895CF93DF93782F882311F4623004
S1130E201CF080E090E040C0209306033093070359
S1130E304093080350930903609305038FB7F89414
S1130E40C82FDD2782B7280F311D411D511D209366
S1130E500A0330930B0340930C0350930D038091CA
S1130E60880390918903A0918A03B0918B038160D8
S1130E708093880390938903A0938A03B0938B0390
S1130E80809156039927AA27BB27281739074A07B1
S1130E905B0738F42093560321BF709342030E94EA
S1130EA0F806CFBF81E090E0DF91CF9108951F92C3
S1130EB00F920FB60F921124FF920F931F932F934B
S1130EC03F934F935F936F937F938F939F93AF93CE
S1130ED0BF93CF93DF93EF93FF93C4B1D5B1D37096
S1130EE0349A379878948FB7F894F82E80919603B3
S1130EF0082F112721E030E0002E02C0220F331FFB
S1130F000A94E2F780916E0390916F0382239323F6
S1130F10892B61F4209530958091D4029091D5026B
S1130F20822393239093D5028093D4024091D402D8
S1130F305091D5024115510511F12091960330913C
S1130F4097032F5F3F4F2C30310511F0C90102C0C8
S1130F5080E090E09C0181E090E0022E02C0880FC6
S1130F60991F0A94E2F784239523892B51F3309334
S1130F70970320939603809196030E940608FFBE70
S1130F800115110569F48FB7F894282F3327D093EE
S1130F904803C093470381E0809366032FBF01C0D9
S1130FA080E099272FB7F8948823C9F461E070E0B2
S1130FB002C0660F771F0A95E2F740916E035091C5
S1130FC06F03CA0186239723892B49F0CB018095AF
S1130FD090954823592350936F0340936E032FBF7A
S1130FE0FF91EF91DF91CF91BF91AF919F918F913D
S1130FF07F916F915F914F913F912F911F910F912D
S1131000FF900F900FBE0F901F901895982F8FB7D9
S1131010F894282F3327E0E7F3E0E90FF11D8081EE
S11310208F7187B92FBF379A369A81E090E008957F
S11310301F93CF93682F80917E03811160958091D7
S1131040AD01482F55274230510509F4ADC0433056
S1131050510524F44115510571F08DC244305105F8
S113106009F469C1443051050CF404C145305105FB
S113107009F4C3C180C220916A038FB7F8949927F9
S11310802093AD028FBF60918003709181036F5FE5
S11310907F4F709381036093800380914C01992763
S11310A08430910559F18530910534F482309105ED
S11310B059F00397B1F06AC08630910509F45EC017
S11310C006970CF44BC062C080918D0290918E0201
S11310D06817790708F44FC283E380936A0383E0B7
S11310E052C08CEC80936A0384E080934C018FEFB0
S11310F09FEF90938103809380033DC2809180038E
S1131100282F332780919102909192022817390752
S1131110F8F4E0916C03F0916D03E60FF71F208162
S113112020936A038091AB029091AC02EDEBF0E066
S11311302927220FF11DE20FF11DC895982F802D4C
S11311403196C89590259093AC028093AB0213C25C
S11311508091AB0280936A0385E015C08091AB0255
S11311609091AC02892F992780936A0386E080933B
S11311704C015093810340938003FDC16430710599
S113118008F4F9C187E080934C01F5C1BB98BA9883
S11311900E94E0061092AB0186E99FE00E942002C3
S11311A0882309F4E8C184C16A3A11F0653571F500
S11311B020919003309191032F5F3F4F309391031F
S11311C02093900380914B03E82FFF27E656FF4FAF
S11311D0849199278217930708F0CDC11092870351
S11311E010929103109290031092D3021092D202A3
S11311F0109293021092AC021092AB0282E290E041
S113120090930F0380930E0384E053C18091AB014C
S1131210882309F4B0C18091450390914603019756
S11312209093460380934503181619060CF4A3C142
S1131230109266038FB7F894C82F2091D40230918E
S1131240D50220FD10C0C90181609093D50280931E
S1131250D4022115310539F4309397032093960372
S113126080E00E940608CFBF109291031092900371
S113127083E01FC16A3A09F449C0653509F446C0E0
S113128080916603882309F476C180914B03E82F8B
S1131290FF27EA54FF4F8491282F33278091470377
S11312A0909148032817390788F561EE80E00E9481
S11312B06E068091CB02682F89E00E946E068AEF49
S11312C090E00197F1F78091B902682F8BE00E94BA
S11312D06E0684E190E00197F1F7BB9ABA9A1092F6
S11312E08103109280031092AC021092AB02109210
S11312F0AD0182E080934C012AEA20936A038FB700
S1131300F89499272093AD028FBF35C10E946A0BD0
S11313108F70907024E230E0829FA001839F500D73
S1131320929F500D1124CA01820F931F909346037C
S113133080934503BDC06A3A11F0653519F4609392
S1131340A80219C1809187039927009721F0039778
S11313500CF04AC006C06093A70249C00E948D0BDE
S113136043C02091A7023091A802922F882790931E
S1131370A8028093A7026093A70210E0220F331FF4
S113138067FD2160660F53E32C3C350749F5E09176
S11313901503F09116034481442301F785E08093FB
S11313A0AD018FB7F894C82F2091D4023091D502A3
S11313B020FD10C0C90181609093D5028093D402AE
S11313C02115310539F43093970320939603842F24
S11313D00E940608CFBF87E0811B8093930207C059
S11313E01F5F183058F203C082E08093AD018091F2
S11313F087038F5F80938703BEC08091A70290917B
S1131400A802982F88279093A8028093A70260933C
S1131410A7022091A7023091A8020090930202C073
S1131420369527950A94E2F7622FE0911503F0911F
S113143016038091D2029091D302E80FF91F208302
S11314404091D2025091D3024F5F5F4F5093D30229
S11314504093D20280910E0390910F0348175907CD
S113146098F58091AB029091AC02EDEBF0E0692726
S1131470660FF11DE60FF11DC895982F802D31964A
S1131480C89590259093AC028093AB0245305105EA
S113149009F071C0E0911503F09116038481992736
S11314A090930F0380930E038E31910528F01482DC
S11314B082E08093AD015FC00097F1F005969093B0
S11314C00F0380930E0357C048175907E1F4809126
S11314D0AB029091AC02EDEBF0E06927660FF11DD1
S11314E0E60FF11DC895982F802D3196C89590254B
S11314F09093AC028093AB0282E290E09093D3028B
S11315008093D20238C044325105A8F1E09115030A
S1131510F091160322A133A18091AB029091AC0209
S11315202817390729F481E090E082A393A302C02D
S113153012A213A20E94A60BC2E0C093AD01E091D7
S11315401503F0911603809147039091480384A3F7
S113155095A38BE19FE00E942002882361F4E0912F
S11315601503F09116038483C093AD0180EC8DB90B
S1131570B8980E94F80681E090E0CF911F910895F9
S1131580CF93C1E020E08FB7F894382F80917D038A
S1131590882391F580919503992781FF08C08AE4F7
S11315A093E09093CE028093CD0280E41AC082FF30
S11315B00FC0E091A501F091A601F093CE02E09353
S11315C0CD0282E48093A8018481992705960DC0F9
S11315D083FF12C08CEA91E09093CE028093CD02F7
S11315E08FEF8093A80181E090E09093AF01809306
S11315F0AE012C2FC0937D033FBF2223F1F08FB7A0
S1131600F894992710924E0110924D0110921103F3
S1131610109210038FBF8EE70E94210BC82F8130D8
S113162061F08FB7F894282F332788E080937D03E7
S11316302FBF86E39BE00E9420028C2F9927CF9135
S11316400895482F8FB7F894282F33279091440397
S113165081E0809344032FBF992319F080E090E048
S113166008954CB95E9A81E090E008958FB7F8949C
S1131670282F332780917D03883011F410927D0345
S11316802FBF8091A80190919503803451F48FB7B6
S1131690F894282F332782E09827909395032FBF3F
S11316A016C08FB7F894282F332784E09827909397
S11316B095032FBFE091A501F091A60114828FB785
S11316C0F89499271092A6011092A5018FBF0E9449
S11316D0C00A08958FB7F894482F552720916303C3
S11316E030916403832F881F8827881F220F331F9C
S11316F0882321F08BE090E1282739272F5F3F4F83
S113170030936403209363038091B1019091B201FB
S1131710282739274FBFC90108958FB7F894382F68
S113172020916B0320FF06C08FB7F8949927DA9AAB
S11317302E7F05C08FB7F8949927DA9821602093FB
S11317406B038FBF3FBF81E090E008956F98B89A14
S1131750C0980E94F80681E090E0089578941F9262
S11317600F920FB60F9211242F933F934F935F93D1
S11317706F937F938F939F93AF93BF93EF93FF9355
S11317808FB7F894282F332780919502882369F026
S1131790809112038093670388608093120383BF50
S11317A08091A60281BF109295022FBF8BEB9FE020
S11317B00E942002FF91EF91BF91AF919F918F9171
S11317C07F916F915F914F913F912F910F900FBE39
S11317D00F901F901895382F80917C0399278230A1
S11317E0910509F46BC0833091052CF4009759F0EE
S11317F0019781F1B7C18330910509F49CC0049726
S113180009F459C1AFC13E3709F0AEC18091490313
S11318109927FC01EE0FFF1FEE0FFF1FE80FF91FC2
S1131820E80FF91FE95AFC4F82819381009709F070
S11318309BC111829093AA028093A90290938C0277
S113184080938B02848195819093690380936803CC
S113185081E085C13E3709F487C180914903992706
S1131860FC01EE0FFF1FEE0FFF1FE80FF91FE80F3B
S1131870F91FE95AFC4F30838091A9029091AA0282
S1131880EDEBF0E0232F2927220FF11DE20FF11DCC
S1131890C895982F802D3196C89590259093AA02CB
S11318A08093A902832F99278134910529F08234EA
S11318B0910509F453C156C182E051C13E3709F480
S11318C051C1609149033D3781F4862F9927FC016A
S11318D0EE0FFF1FEE0FFF1FE80FF91FE80FF91FB0
S11318E0E95AFC4F80E281833FC1862F9927FC018E
S11318F0EE0FFF1FEE0FFF1FE80FF91FE80FF91F90
S1131900E95AFC4F2181232721838091A9029091D8
S1131910AA02EDEBF0E02927220FF11DE20FF11DE1
S1131920C895982F802D3196C89590259093AA023A
S11319308093A90213C140918B0250918C024C32C6
S1131940510508F0BAC03D3711F484E008C13E37B0
S113195009F07FC04230510508F45FC0E09168038C
S1131960F0916903E40FF51F82919927382F2227FC
S113197082919927282B392B8091A9029091AA0250
S11319806091490328173907E1F4862F9927FC0150
S1131990EE0FFF1FEE0FFF1FE80FF91FE80FF91FEF
S11319A0E95AFC4F425050404283538387E790E109
S11319B00E942002809149038F5F817080934903C4
S11319C010C0862F9927FC01EE0FFF1FEE0FFF1F9B
S11319D0E80FF91FE80FF91FE95AFC4F128213822E
S11319E01182809149039927FC01EE0FFF1FEE0F2E
S11319F0FF1FE80FF91FE80FF91FE95AFC4F828116
S1131A009381892BD9F48481958190936903809380
S1131A10680381E080937C0313C080914903992774
S1131A20FC01EE0FFF1FEE0FFF1FE80FF91FE80F79
S1131A30F91FE95AFC4F12821382118210927C031F
S1131A401092AA021092A90210928C0210928B0298
S1131A508BC0E0916803F0916903E40FF51F3083B4
S1131A6040918B0250918C0242305105E8F0209154
S1131A70A9023091AA02E0916803F0916903E40F8E
S1131A80F51F32978081EDEBF0E08327880FF11D7D
S1131A90E80FF11DC895322F202D3196C8953025B9
S1131AA03093AA022093A9024F5F5F4F50938C0298
S1131AB040938B0259C03E37D1F41092AA0210927F
S1131AC0A90210928C0210928B02809149039927EB
S1131AD0FC01EE0FFF1FEE0FFF1FE80FF91FE80FC9
S1131AE0F91FE95AFC4F1282138211823BC080E233
S1131AF08327E0916803F091690320918B02309170
S1131B008C02E20FF31F808340918B0250918C0270
S1131B1042305105E8F02091A9023091AA02E091E7
S1131B206803F0916903E40FF51F32978081EDEBB0
S1131B30F0E08327880FF11DE80FF11DC895322FBF
S1131B40202D3196C89530253093AA022093A902FE
S1131B504F5F5F4F50938C0240938B0283E08093DE
S1131B607C0302C010927C0381E090E008951F93EF
S1131B70CF93E091D002F091D1028091020183834E
S1131B80E091D002F091D10211E08FB7F894C82F00
S1131B908091A901882311F010E018C01093A901C5
S1131BA0F0936D03E0936C038481992705969093D9
S1131BB09202809391020E946A0B8F7790708496B0
S1131BC090934603809345031093AB01CFBF112339
S1131BD009F453C08FB7F89499272091AD018FBFB2
S1131BE0263009F04AC040918803509189036091DE
S1131BF08A0370918B0340FF17C08FB7F894282F86
S1131C003327DB01CA018E7F809388039093890375
S1131C10A0938A03B0938B032FBF0097A105B1054E
S1131C2019F481E0809342036BE380E00E946E0626
S1131C3080ED97E00197F1F769E380E00E946E067A
S1131C4088EC90E00197F1F70E94E006BB98BA98FF
S1131C5080EC8DB9B8980E94F80620E230E040E0AC
S1131C6050E061E080E00E940A078FB7F894282FC3
S1131C70332782E08093AD012FBF112339F48FB74E
S1131C80F8949927109286038FBF02C00E948D0B8F
S1131C90CF911F9108958FB7F89499272091440309
S1131CA0109244038FBF222309F4A4C080917D03C2
S1131CB0873031F410927D0386E39BE00E9420027A
S1131CC021E080917D0399278430910509F46EC049
S1131CD08530910554F48230910561F1833091058A
S1131CE00CF058C0019749F07CC08630910509F486
S1131CF071C006970CF463C074C082E080937D03C6
S1131D0020914D0130914E018091A801EDEBF0E05E
S1131D108327880FF11DE80FF11DC895322F202D60
S1131D203196C895302530934E0120934D01809112
S1131D30A80154C0E091CD02F091CE02209110038D
S1131D4030911103E20FF31F508180914D01909166
S1131D504E01EDEBF0E0452F4927440FF11DE40F50
S1131D60F11DC895982F802D3196C8959025909394
S1131D704E0180934D012F5F3F4F30931103209309
S1131D8010038091AE019091AF012817390798F0A4
S1131D9084E00FC08091820390E289270E94210B86
S1131DA0282F8091650380937D031BC050914D01C2
S1131DB085E080937D03852F0E94FD0E11C08091E4
S1131DC04D0190914E01292F332786E080937D03A6
S1131DD0822FF2CF87E080937D038EE70E94210B50
S1131DE0282F213039F088E080937D0386E39BE03F
S1131DF00E94200281E090E00895982F8D57823050
S1131E0078F48FB7F894282F332780917D0380933B
S1131E10650383E080937D03909382032FBF9DE746
S1131E20892F0E94210B992708958FBF08958FB79A
S1131E30F89499270895CF93DF938FB7F894682F78
S1131E407727A0911503B091160397961D921C92C3
S1131E50989794968D919C9195979C01220F331F8E
S1131E60220F331F280F391F40910203509103039F
S1131E70CA01880F991F840F951F280F391FC3E0CB
S1131E8036952795CA95E1F730930303209302030F
S1131E906FBF92968D919C919397892B69F11396BC
S1131EA09C91139780910201981711F09D0126C00F
S1131EB08FB7F894282F90918503E92FFF27EE0F11
S1131EC0FF1FE45BFC4FC081D1818C81882351F4D6
S1131ED0A083B1839F5F892F65E00E945412909381
S1131EE0850302C0C0E0D0E02FBF209729F080E036
S1131EF091E10E94200201C0ED019E018FB7F89488
S1131F0099272115310521F03093160320931503E9
S1131F10E0911503F091160314828FBF80EC8DB904
S1131F20B8980E94F806DF91CF9108958FB7F8947E
S1131F309927E0916C03F0916D0317A210A68FBF4F
S1131F408091860381FF05C08AE491E10E9420020A
S1131F500BC08FB7F8949927E091D002F091D10289
S1131F601482109286038FBF8FB7F894992710922A
S1131F70A9018FBF0895CF93DF9381E0809342033B
S1131F808091880390918903A0918A03B0918B0377
S1131F900097A105B10509F46DC0FD01EC0180FFB6
S1131FA069C08091560399270196AA2797FDA095A9
S1131FB0BA2F20910A0330910B0340910C035091E6
S1131FC00D03281B390B4A0B5B0B20930A03309338
S1131FD00B0340930C0350930D032330310541054B
S1131FE051050CF047C0809105038823A9F4809122
S1131FF0060390910703A0910803B0910903280FE9
S1132000391F4A1F5B1F20930A0330930B0340932D
S11320100C0350930D0314C081E090E080959095DB
S1132020AA2797FDA095BA2F8C239D23AE23BF2307
S11320308093880390938903A0938A03B0938B03BE
S113204080919203882319F48FEF809392039091E7
S113205092039F5F90939203809194028F5F809389
S11320609402E92FFF27E655FE4F108281E891E1A3
S11320700E9420020E94A701DF91CF91089587B7A3
S113208099278C7F009719F080E090E01AC06F992F
S113209018C0379B03C088E090E013C087B7992726
S11320A083709070892B59F081B792B7891B803166
S11320B018F48CE190E005C088E190E002C080E172
S11320C090E0382F25B7237E8C3121F0883111F030
S11320D008C0000080B7992787709070892BC9F7D2
S11320E0237E232B25BF85B7806285BF0895EF9299
S11320F0FF920F931F93CF93DF9390917F0386E01A
S1132100989F7001112487E593E0E80EF91EF7010A
S1132110C481D58182819381059708F456C02081BA
S1132120822F99278134910561F0823491052CF432
S11321308034910509F449C042C082349105D9F034
S11321403EC081E090E08AA39BA3F70121818FB771
S1132150F8949091860390FD18C00091D0021091DC
S1132160D102936090938603D093D102C093D0029E
S11321702093D60218C081E090E08AA39BA38FB776
S1132180F8949091860390FF03C000E010E00BC028
S11321900091D0021091D102916090938603D09364
S11321A0D102C093D0028FBF0115110511F48E0125
S11321B004C087EB9DE00E942002E80106C0209342
S11321C0AC0188E292E10E9420028FB7F894282F94
S11321D03327209719F0F701C483D583F7011282BE
S11321E01382118280917F038F5F817080937F03BC
S11321F02FBFDF91CF911F910F91FF90EF90089522
S1132200CF93DF938FB7F894282F3327809114034B
S1132210E82FFF27EE0FFF1FE45BFC4FC081D18145
S11322208F5F65E00E945412909314032FBF21E046
S11322308FB7F8949091950392FD08C094609093A1
S11322409503D093A601C093A50101C020E08FBFE0
S1132250213019F40E94C00A282F213011F01C8269
S113226016C08FB7F894382F20916B0321FF06C056
S11322708FB7F8949927D99A2D7F05C08FB7F89412
S11322809927D998226020936B038FBF3FBFDF91BA
S1132290CF9108952091D60231E08FB7F8949091B0
S11322A0950391FD06C092609093950320934A0391
S11322B001C030E08FBF313011F40E94C00A8FB7E3
S11322C0F894382F20916B0322FF06C08FB7F8943F
S11322D09927D89A2B7F05C08FB7F8949927D89857
S11322E0246020936B038FBF3FBF8FB7F894992767
S11322F0E091D002F091D1021482109286038FBF34
S11323000895EF92FF921F93CF93DF9390919402DD
S1132310992321F451E0E52EF12C16C08091A701F8
S1132320882319F48FEF8093A7018091A7018F5F11
S11323308093A701915090939402E82FFF27E655CC
S1132340FE4F8081E82EFF24EE2009F07BC0E0914F
S11323504B03EE2309F476C08FB7F89499272091A4
S1132360AD011091AB018FBF33272230310521F02D
S11323702630310591F15EC08E2F9927880F991F61
S1132380FC01EF55FF4F24913327D22FCC278E55D4
S11323909F4FFC0184919927C82BD92B112309F055
S11323A049C08FB7F894282F332786E08093AD0176
S11323B02FBFCE01AA27BB279C01AD0161E0812F6D
S11323C00E940A07612F8BE00E946E066FE3812F43
S11323D00E946E060E94A60B35C0FF27E155FF4FF1
S11323E08491C82FDD278FB7F894282F332782E0F4
S11323F08093AD012FBF6BE38E2D0E946E0680ED9E
S113240097E00197F1F769E38E2D0E946E0688EC40
S113241090E00197F1F7BB98BA980E94E00680EC2F
S11324208DB9B8980E94F806CE01AA27BB279C0153
S1132430AD0104C020E230E040E050E061E080E023
S11324400E940A07DF91CF911F91FF90EF900895AA
S11324508FB7F894282F3327809195038860809351
S113246095032FBF0E94C00A0895629FD001739FF5
S1132470F001829FE00DF11D649FE00DF11D929F1C
S1132480F00D839FF00D749FF00D659FF00D99275B
S1132490729FB00DE11DF91F639FB00DE11DF91F7F
S11324A0BD01CF0111240895991B79E004C0991F3F
S11324B0961708F0961B881F7A95C9F7809508959A
S11324C0A1E21A2EAA1BBB1BFD010DC0AA1FBB1F34
S11324D0EE1FFF1FA217B307E407F50720F0A21BA6
S11324E0B30BE40BF50B661F771F881F991F1A9413
S11324F069F760957095809590959B01AC01BD013D
S1072500CF01089566
S1132504010033008025009224200000201C0000D8
S1132514001900008016005D74140000C01200C588
S11325244E110049121000BD04880552061C07E62A
S113253407B0087B09450A0F0BAA01F10138028090
S10F254402C7020E0355039C03E30301CD
S9030000FC
